:100000000C9462000C9477040C944F040C948A00B6
:100010000C948A000C948A000C948A000C948A0038
:100020000C948A000C948A000C948A000C948A0028
:100030000C948A000C948A000C948A000C948A0018
:100040000C9405040C948A000C94D3030C94AD0317
:100050000C948A000C948A000C948A000C948A00F8
:100060000C948A000C948A000000000024002700F1
:100070002A0000000000250028002B0000000008D6
:10008000000201000003040700000000000000005F
:10009000010204081020408001020408102001021F
:1000A000040810200000000023002600290004049A
:1000B0000404040404040202020202020303030310
:1000C0000303060511241FBECFEFD8E0DEBFCDBF6E
:1000D00023E0AEE1B2E001C01D92AE31B207E1F71C
:1000E00012E0A0E0B1E0E2EEF5E102C005900D9271
:1000F000AE31B107D9F710E0C2E6D0E004C02197D5
:10010000FE010E94BF09C136D107C9F70E94D80578
:100110000C94EF0A0C940000AF92BF92CF92DF9242
:10012000EF92FF920F931F93CF93DF936C017B01AC
:100130008B01040F151FEB015E01AE18BF08C0173D
:10014000D10759F06991D601ED91FC910190F081B0
:10015000E02DC6010995892B79F7C501DF91CF9173
:100160001F910F91FF90EF90DF90CF90BF90AF90D5
:100170000895FC01538D448D252F30E0842F90E0AD
:10018000821B930B541710F0CF9608950197089592
:10019000FC01918D828D981761F0A28DAE0FBF2F5B
:1001A000B11D5D968C91928D9F5F9F73928F90E0B1
:1001B00008958FEF9FEF0895FC01918D828D981720
:1001C00031F0828DE80FF11D858D90E008958FEF5D
:1001D0009FEF0895FC01918D228D892F90E0805C26
:1001E0009F4F821B91098F739927089583E392E0B3
:1001F0000E94EA0021E0892B09F420E0822F089573
:1002000083E392E00E94EA00892BD1F083E392E03D
:100210000E94C8008C3329F410921F0210921E0213
:10022000EFCF8A30C9F380911E0290911F0284366D
:10023000910594F7019690931F0280931E02E0CFE0
:1002400008950E94F60081110C9400010895FC01AC
:10025000A48DA80FB92FB11DA35ABF4F2C91848D27
:1002600090E001968F739927848FA689B7892C9384
:10027000A089B1898C91837080648C93938D848DD7
:10028000981306C00288F389E02D80818F7D8083DA
:100290000895EF92FF920F931F93CF93DF93EC019A
:1002A00081E0888F9B8D8C8D98131AC0E889F9891D
:1002B000808185FF15C09FB7F894EE89FF89608320
:1002C000E889F98980818370806480839FBF81E0A1
:1002D00090E0DF91CF911F910F91FF90EF900895E3
:1002E000F62E0B8D10E00F5F1F4F0F731127E02EBE
:1002F0008C8D8E110CC00FB607FCFACFE889F989F6
:10030000808185FFF5CFCE010E942701F1CFEB8DD3
:10031000EC0FFD2FF11DE35AFF4FF0829FB7F894C9
:100320000B8FEA89FB8980818062CFCFCF93DF93E7
:10033000EC01888D8823B9F0AA89BB89E889F989FD
:100340008C9185FD03C0808186FD0DC00FB607FC32
:10035000F7CF8C9185FFF2CF808185FFEDCFCE0165
:100360000E942701E9CFDF91CF910895833081F07A
:1003700028F4813099F08230A9F008958730A9F0EF
:100380008830C9F08430B1F4809180008F7D03C043
:10039000809180008F7780938000089584B58F7757
:1003A00084BD089584B58F7DFBCF8091B0008F7799
:1003B0008093B00008958091B0008F7DF9CF1F9396
:1003C000CF93DF93282F30E0F901E458FF4F849159
:1003D000F901E057FF4FD491F901E255FF4FC49165
:1003E000CC23A9F0162F81110E94B601EC2FF0E06A
:1003F000EE0FFF1FEE58FF4FA591B4918FB7F89401
:10040000EC91111108C0D095DE23DC938FBFDF91F2
:10041000CF911F910895DE2BF8CFCF93DF9390E01B
:10042000FC01E057FF4F249182559F4FFC018491BE
:100430008823C9F090E0880F991FFC01E859FF4F0D
:10044000A591B491FC01EE58FF4FC591D491611173
:100450000DC09FB7F8948C91209582238C9388814E
:10046000282328839FBFDF91CF910895623051F4F4
:100470009FB7F8943C91822F809583238C93E881D9
:100480002E2BEFCF8FB7F894EC912E2B2C938FBFA0
:10049000EACF3FB7F8948091250290912602A0916F
:1004A0002702B091280226B5A89B05C02F3F19F05E
:1004B0000196A11DB11D3FBFBA2FA92F982F8827E4
:1004C000BC01CD01620F711D811D911D42E0660FBF
:1004D000771F881F991F4A95D1F708958F929F9291
:1004E000AF92BF92CF92DF92EF92FF924B015C01ED
:1004F0000E9449026B017C010E9449026C197D092E
:100500008E099F09683E734081059105A8F321E09B
:10051000821A9108A108B10888EEC80E83E0D81E9F
:10052000E11CF11C81149104A104B10429F7FF908E
:10053000EF90DF90CF90BF90AF909F908F900895F5
:100540002FB7F894609121027091220280912302CA
:10055000909124022FBF0895FC01848187FD05C07E
:1005600091E0692763830E94DF0180E00895FC0128
:10057000808580FD04C082FB882780F9089580E093
:100580000895FC019085957081E0953009F080E038
:100590000895862F642F0C940D02CF93DF93FC01F6
:1005A000218530E0F901E458FF4F8491F901E057CB
:1005B000FF4FD491F901E255FF4FC491CC2379F05C
:1005C00081110E94B601EC2FF0E0EE0FFF1FEC55F9
:1005D000FF4FA591B491EC91ED2381E009F480E007
:1005E0008170DF91CF910895DC01ED91FD918081C3
:1005F000ED91FD919081ED91FD916C9163708E2351
:1006000009F064609F2309F06860E1E1F3E0E60F20
:10061000F11D659565956D936D917D918D919D9180
:10062000099423C01AC012C016C010C01EC009C051
:1006300014C013C006C019C009C00DC007C00DC04A
:1006400014C062507040804090400BC061507040B8
:100650008040904006C06E5F01C06F5F7F4F8F4F3C
:100660009F4F9E938E937E936E9308958091FB028D
:10067000823078F4F89480EF92E00E94F402609166
:10068000F7027091F8028091F9029091FA02789441
:100690000895F894F4CF8F929F92AF92BF920F93E8
:1006A0001F93CF93DF93CDB7DEB7A1970FB6F89422
:1006B000DEBF0FBECDBF19A2423008F44AE08E0162
:1006C0000F5D1F4F842E912CB12CA12CA5019401FC
:1006D0000E947E09E62FB901CA01EA3044F5E05DC7
:1006E000D801EE938D01232B242B252B79F790E055
:1006F00080E0109769F0FD0101900020E9F7319743
:10070000AF014A1B5B0BBD0183E392E00E948C00AA
:10071000A1960FB6F894DEBF0FBECDBFDF91CF918B
:100720001F910F91BF90AF909F908F900895E95CBB
:10073000D7CF009769F0FC0101900020E9F73197CD
:10074000AF01481B590BBC0183E392E00C948C0071
:1007500090E080E008950E94EA0A1F920F920FB67F
:100760000F9211242F933F934F935F936F937F9337
:100770008F939F93AF93BF93EF93FF9383E392E0A5
:100780000E942701FF91EF91BF91AF919F918F91AF
:100790007F916F915F914F913F912F910F900FBE7D
:1007A0000F901F9018951F920F920FB60F92112461
:1007B0002F938F939F93EF93FF93E0914302F091D8
:1007C00044028081E0914902F0914A0282FD1BC0FF
:1007D000908180914C028F5F8F7320914D02821720
:1007E00041F0E0914C02F0E0ED5CFD4F958F80937D
:1007F0004C02FF91EF919F918F912F910F900FBE1F
:100800000F901F9018958081F4CF1F920F920FB612
:100810000F9211242F933F938F939F93AF93BF9386
:100820008091210290912202A0912302B091240292
:100830003091200223E0230F2D3758F50196A11D9A
:10084000B11D209320028093210290932202A09355
:100850002302B09324028091250290912602A09158
:100860002702B09128020196A11DB11D8093250297
:1008700090932602A0932702B0932802BF91AF91D4
:100880009F918F913F912F910F900FBE0F901F90CE
:10089000189526E8230F0296A11DB11DD2CF1F92F5
:1008A0000F920FB60F9211242F933F934F935F93A4
:1008B0006F937F938F939F93AF93BF93EF93FF9328
:1008C0008091D2029091D3020E94F402FF91EF91A5
:1008D000BF91AF919F918F917F916F915F914F9158
:1008E0003F912F910F900FBE0F901F9018951F9260
:1008F0000F920FB60F9211242F933F934F935F9354
:100900006F937F938F939F93AF93BF93EF93FF93D7
:100910008091D0029091D1020E94F402FF91EF9158
:10092000BF91AF919F918F917F916F915F914F9107
:100930003F912F910F900FBE0F901F901895CF925F
:10094000DF92EF92FF920F931F93CF93DF93EC010F
:10095000E62E84E090E00E94C509FC0184E68083D5
:1009600085E6818386E6828387E683838CE291E055
:10097000998388838FEF8A838B838C838A878B8785
:100980008C8784E089878F016E0185E0C80ED11CB9
:10099000F12CF80181918F0187FD36C0F60181931A
:1009A0006F0161E00E940D02F394F4E0FF12F1CFB9
:1009B0008FEF8C8382E391E0998388838B8587FD19
:1009C00011C0282F082E000C330BE216130651F02D
:1009D0009A85913019F460E00E94DF0160E08B8518
:1009E0000E940D0282E08A87EB8662E08E2D0E94D3
:1009F0000D0281E08C87DF91CF911F910F91FF90C5
:100A0000EF90DF90CF900895F986D2CFCF93DF9308
:100A1000109236021092350288EE93E0A0E0B0E02A
:100A20008093370290933802A0933902B0933A0230
:100A300088E391E0909334028093330285EC90E058
:100A40009093400280933F0284EC90E090934202A6
:100A50008093410280EC90E09093440280934302A3
:100A600081EC90E0909346028093450282EC90E006
:100A7000909348028093470286EC90E090934A025C
:100A80008093490210924C0210924D0210924E0235
:100A900010924F0262E68DE093E00E949F0463E6AD
:100AA00080E093E00E949F0462E08AE00E940D02D1
:100AB00062E089E00E940D02E8EBF0E0E491F0E0F2
:100AC000EE0FFF1FEC55FF4FA591B491B093F102CB
:100AD000A093F002EAE9F0E044914093F402E7EBDE
:100AE000F0E0E491F0E0EE0FFF1FEC55FF4FC591F1
:100AF000D491D093F302C093F202E9E9F0E0E491DB
:100B0000E093F5021092F7021092F8021092F902A7
:100B10001092FA022BE33FE1C9010197F1F79C9192
:100B2000842F892391E009F490E08881E82309F07B
:100B300092609093F6021092FB028EE491E0909303
:100B4000FD028093FC0289E591E09093FF0280937F
:100B5000FE022AE431E03093D5022093D4021092B1
:100B6000D6021092D7021092D8021092D9028AE0CF
:100B700090E09093DB028093DA021092DC021092F4
:100B8000DD023093E3022093E2021092E40210921D
:100B9000E5021092E6021092E7029093E902809338
:100BA000E8021092EA021092EB02DF91CF910895D1
:100BB000CF93DF9300D000D0CDB7DEB7789484B563
:100BC000826084BD84B5816084BD85B5826085BD49
:100BD00085B5816085BD80916E00816080936E00D7
:100BE00010928100809181008260809381008091C9
:100BF000810081608093810080918000816080937A
:100C000080008091B10084608093B1008091B00039
:100C100081608093B00080917A00846080937A0034
:100C200080917A00826080937A0080917A0081605E
:100C300080937A0080917A00806880937A00109285
:100C4000C10024ED32E03C832B8300E211E06AE036
:100C5000C62ED12CD801FC9011967C91AB81BC8121
:100C6000ED91FC9111970280F381E02D42E050E07C
:100C70006F2DCD010995EB81FC81F1861086DF0196
:100C80000190F081E02D0190F081E02DCD010995DA
:100C9000882329F0EB81FC818085836080870E9416
:100CA000A002AB81BC8112966D937D938D939C9332
:100CB00015971796DC92CE9216970C5F1F4F1E96D3
:100CC000BC83AB83A05FB24029F60E9436036093D9
:100CD0002F0270933002809331029093320261E0D0
:100CE0008CE00E940D0261E08CE00E94DF0168EE62
:100CF00073E080E090E00E946E02E0914302F09188
:100D0000440282E08083E0913F02F0914002108231
:100D1000E0914102F091420280E1808310924B0207
:100D2000E0914702F091480286E08083E09145021D
:100D3000F0914602808180618083E0914502F091CC
:100D40004602808188608083E0914502F0914602EE
:100D5000808180688083E0914502F0914602808125
:100D60008F7D808382E390E0A0E0B0E08093370243
:100D700090933802A0933902B0933A0284E691E04E
:100D8000F1E086379F0709F467C021E029838C587A
:100D9000914009F0198254E6652E51E0752E0E94AB
:100DA000A0024B015C018091160190911701A09166
:100DB0001801B0911901AC01BD014854544F6F4F57
:100DC0007F4F84169506A606B70628F4881699065E
:100DD000AA06BB0678F582EA91E00E94990384E6B0
:100DE00091E00E94990381EB91E00E9499034AE00F
:100DF00063E070E080E090E00E944B0381EB91E0C3
:100E00000E94990380E191E00E9499038DEE91E0A8
:100E10000E9499038092160190921701A0921801E6
:100E2000B092190180920C0190920D01A0920E01D6
:100E3000B0920F01B1E0BA83EFEE6E16E1E07E06EC
:100E400009F01A828091FC029091FD02F2E082305A
:100E50009F0729F421E013C041E049839CCF835BC5
:100E60009140C1F38091FE029091FF0221E0B1E038
:100E70008E3B9B0721F0895C914009F020E02A809D
:100E8000222009F4FCC0222309F4F9C00E94360391
:100E900024E030E040E050E00E94A00969017A01BE
:100EA00080912F0290913002A0913102B0913202D4
:100EB0008C159D05AE05BF050CF0E8C08091FE02C3
:100EC0009091FF020E9499038DEE91E00E94990398
:100ED00080920C0190920D01A0920E01B0920F0130
:100EE000C0922F02D0923002E0923102F092320290
:100EF00040E2E42E41E0F42E24ED32E03C832B83EB
:100F0000D12CC12CAB81BC8118968C9118978B7F0A
:100F100018968C931897ED91FC9111970190F081A0
:100F2000E02DCD010995182FEB81FC8180858695F8
:100F30008170181709F4B5C00E94A002AB81BC8172
:100F400012966D937D938D939C93159718968C9123
:100F5000B2E08B27EB81FC8180878B819C810E9492
:100F6000B702811107C08B819C810E94C102882336
:100F700009F474C021E0F4ED6F16F1E07F0609F08A
:100F800020E0D7010D911C91C8010397039708F445
:100F9000C6C081E00431110509F080E0222311F080
:100FA000811111C0C8014397039708F4BAC081E0CA
:100FB0000C31110509F080E02980222009F4B3C02A
:100FC000882309F4B0C08092080190920901A09290
:100FD0000A01B0920B0110922E0210922D02D7013D
:100FE00012968D919C910E9499038B819C810E9405
:100FF000B702882309F46EC187EE91E00E9499033D
:101000000B321105E9F42A802220D1F080912902C7
:1010100090912A02009709F054C144244394512C22
:1010200050922A024092290280920001909201017E
:10103000A0920201B092030161E080E00E94DF0112
:1010400064E670E080E090E00E946E0280920C0105
:1010500090920D01A0920E01B0920F012B813C8164
:10106000225F3F4F3C832B8334E0E30EF11CCA9494
:10107000CD2809F489C0CC24C394D12C43CF0E943D
:10108000360322E030E040E050E006CFC816D90633
:10109000EA06FB060CF024CF8091FC029091FD0241
:1010A00011CF0E94A002AB81BC8112962D913D917F
:1010B0004D915C9115971B012C01221A330A440AA9
:1010C000550AB201A10116968D919C91B0E0A0E065
:1010D000481759076A077B0708F43FCFAB81BC81EB
:1010E00018968C918170181709F437CF0E94A002CE
:1010F000EB81FC8162837383848395838085F1E037
:101100008F278460AB81BC8118968C930E94A002CB
:10111000EB81FC8162877387848795871ECF81E08E
:101120003DCF81E049CF0231110511F4211108C0F2
:101130000A31110509F053CF3980332009F44FCF1C
:101140008091080190910901A0910A01B0910B01D1
:1011500086509F4FAF4FBF4F88169906AA06BB0611
:1011600098F044244394512C50922E0240922D0228
:10117000D0922C02C0922B02809204019092050121
:10118000A0920601B09207018FEE681681E0780602
:1011900001F58091000190910101A0910201B091AF
:1011A000030188539D4CAF4FBF4F88159905AA0581
:1011B000BB0520F410922A02109229028091290284
:1011C00090912A0260E0892B09F061E080E00E94A2
:1011D000DF0180910C0190910D01A0910E01B09161
:1011E0000F01AC01BD014C595F4F6F4F7F4F84160B
:1011F0009506A606B70628F488169906AA06BB0621
:1012000060F48DEE91E00E94990380920C0190921F
:101210000D01A0920E01B0920F01809104019091F6
:101220000501A0910601B091070186509F4FAF4F75
:10123000BF4F88159905AA05BB05D8F580912D02E9
:1012400090912E020197A9F5E0912B02F0912C02CA
:10125000EE0FFF1FEE0FFF1FE05EFE4F82819381B6
:101260000E94990380912B0290912C02AEE0A89FDE
:101270008001A99F100D11240C521D4FC8010E941E
:10128000B702882399F187EE91E00E94990364E602
:1012900070E080E090E00E946E0280920C019092DB
:1012A0000D01A0920E01B0920F0110922E02109229
:1012B0002D020E94F600882309F471CD0E940001DE
:1012C0006ECD019709F0BCCE10922A02109229022D
:1012D00060E0B3CE8B819C810E94C102882309F417
:1012E000AFCE8BEE91E00E949903AACEC8010E9476
:1012F000C102882361F28BEE91E0C7CFA1E21A2EE2
:10130000AA1BBB1BFD010DC0AA1FBB1FEE1FFF1FA9
:10131000A217B307E407F50720F0A21BB30BE40BF9
:10132000F50B661F771F881F991F1A9469F7609540
:101330007095809590959B01AC01BD01CF010895FA
:10134000052E97FB1EF400940E94B70957FD07D0A5
:101350000E947E0907FC03D04EF40C94B709509507
:101360004095309521953F4F4F4F5F4F0895909591
:101370008095709561957F4F8F4F9F4F0895EE0F29
:10138000FF1F0590F491E02D09940F931F93CF93C5
:10139000DF938230910510F482E090E0E0911C032D
:1013A000F0911D0330E020E0B0E0A0E0309799F428
:1013B0002115310509F44AC0281B390B24303105A9
:1013C000D8F58A819B816115710589F1FB019383B1
:1013D0008283FE0111C0408151810281138148172F
:1013E0005907E0F04817590799F4109761F01296E1
:1013F0000C93129713961C933296CF01DF91CF91E5
:101400001F910F91089500931C0310931D03F4CFB7
:101410002115310551F04217530738F0A901DB01BE
:101420009A01BD01DF01F801C1CFEF01F9CF90931F
:101430001D0380931C03CDCFFE01E20FF31F8193A8
:1014400091932250310939832883D7CF20911A03F1
:1014500030911B03232B41F420911C0130911D017D
:1014600030931B0320931A0320911A0130911B0122
:101470002115310541F42DB73EB740911E01509121
:101480001F01241B350BE0911A03F0911B03E21797
:10149000F307A0F42E1B3F0B2817390778F0AC0197
:1014A0004E5F5F4F2417350748F04E0F5F1F509374
:1014B0001B0340931A03819391939FCFF0E0E0E0E8
:1014C0009CCFCF93DF930097E9F0FC013297138212
:1014D0001282A0911C03B0911D03ED0130E020E0C9
:1014E0001097A1F420813181820F931F20911A035C
:1014F00030911B032817390709F061C0F0931B03D3
:10150000E0931A03DF91CF910895EA01CE17DF0728
:10151000E8F54A815B819E0141155105B1F7E9016A
:10152000FB83EA8349915991C40FD51FEC17FD073E
:1015300061F4808191810296840F951FE90199835E
:101540008883828193819B838A83F0E0E0E0129616
:101550008D919C9113970097B9F52D913C9111971E
:10156000CD010296820F931F20911A0330911B0325
:101570002817390739F6309751F510921D0310924C
:101580001C03B0931B03A0931A03BCCFD383C28365
:1015900040815181840F951FC817D90761F44E5FB0
:1015A0005F4F88819981480F591F518340838A81F9
:1015B0009B81938382832115310509F0B0CFF0938D
:1015C0001D03E0931C039ECFFD01DC01C0CF1382FD
:1015D0001282D7CF81E090E0F8940C94EF0AF8944F
:0215E000FFCF3B
:1015E200FFFFFFFFFFFFFFFFFFFFFFFFFFFFFFFF09
:1015F200322E362E3400FFFFFFFF00001E03800054
:101602000B000D020D00150200000000AB030000EC
:101612000000AC020000000049018C00B9009601F4
:10162200EA00C800DC0000000000CD02C902454EFD
:10163200435F53454C5F444E00454E435F53454C18
:101642005F5550005265616C53696D476561722D3B
:101652004735415454005265616C53696D47656169
:10166200722D473130303050464431005265616C42
:1016720053696D476561722D47313030304D4644B4
:101682003100232323235265616C53696D476561E1
:10169200722300454E435F414C545F555000454E06
:1016A200435F4844475F444E00454E435F414C54BC
:1016B2005F444E005265616C53696D476561722DDE
:1016C200474D41333530003D310A003D300A00526A
:1016D20065616C53696D476561722D4746433530CC
:1016E2003000454E435F4844475F55500042544ED8
:0E16F2005F53454C0042544E5F50575200006B
:00000001FF
